S01C000064656D6F70726F675F656B5F6C6D3373383936322E73726563C5
S113800058040020E59B0000C39B0000C39B0000B4
S1138010C39B0000C39B0000C39B0000C39B0000E4
S1138020C39B0000C39B0000C39B0000C39B0000D4
S1138030C39B0000C39B0000C39B000097920000F9
S1138040C39B0000C39B0000C39B0000C39B0000B4
S1138050C39B0000C39B0000C39B0000C39B0000A4
S1138060C39B0000C39B0000C39B0000C39B000094
S1138070C39B0000C39B0000C39B0000C39B000084
S1138080C39B0000C39B0000C39B0000C39B000074
S1138090C39B0000C39B0000C39B0000C39B000064
S11380A0C39B0000C39B0000C39B0000C39B000054
S11380B0C39B0000C39B0000C39B0000C39B000044
S11380C0C39B0000C39B0000C39B0000C39B000034
S11380D0C39B0000C39B0000C39B0000C39B000024
S11380E0C39B0000C39B0000C39B0000C39B000014
S10780F0EE11AA558A
S11380F4DFF85017884207D0DFF84C17884203D0C2
S1138104DFF84817884201D1012000E00020C0B202
S11381147047DFF83017884208D0DFF82C178842FC
S113812406D0DFF82817884204D005E0372005E09C
S1138134382003E0392001E05FF0FF30704770B568
S113814482B00500280B0003FFF7E3FF040014F1D9
S1138154010F04D1F921DFF8F80600F095FBDFF8EC
S1138164F406006801212200303A914011EA000625
S1138174002E02D0200000F0CAFB286800200090E2
S113818402E00098401C009000980528F9DB2D6853
S1138194002E02D0200000F079FB280076BD81B0C7
S11381A401600020009002E00098401C00900098B8
S11381B40528F9DB01B07047F8B504000D0016007A
S11381C400270BE0E15D7F1CB74203DAE05D51EA6E
S11381D400217F1C2800FFF7E2FF2D1DB742F1DBCD
S11381E4F1BDF8B504000D00160000270AE02800CC
S11381F4FFF7A5FF2D1DE0557F1CB74202DA000AE4
S1138204E0557F1CB742F2DBF1BD38B50400200011
S1138214FFF76EFF002805D140F2D911DFF83006CC
S113822400F032FB01212000FFF7B9FF14F1200014
S1138234FFF785FF0004F9D4B02114F12400FFF7FB
S1138244AEFF002114F13400FFF7A9FF002114F15B
S11382543800FFF7A4FF01250BE014F12000FFF719
S11382646EFF0004F9D4290014F12000FFF797FFEE
S11382746D1C212DF1DB0C2114F12400FFF78FFF79
S113828401250BE014F12000FFF759FF0004F9D491
S1138294290014F12000FFF782FF6D1C212DF1DB6E
S11382A4201DFFF74CFF31BD10B504002000FFF77B
S11382B41FFF002805D140F23A21DFF8940500F0AD
S11382C4E3FA2000FFF73BFF410849002000FFF7D1
S11382D466FF10BD70B504000D002000FFF708FF11
S11382E4002805D14FF45971DFF8640500F0CCFA85
S11382F4002D05D140F26531DFF8540500F0C4FACD
S11383042868801E0F2805D340F26B31DFF840053E
S113831400F0BAFA6868002802D06868092805D30E
S11383244FF45C71DFF8280500F0AEFAA868002861
S113833402D0A868052805D340F27531DFF810058A
S113834400F0A2FAE868B0F5806F02D8E868002863
S113835405D140F27B31DFF8F80400F095FA2000EF
S1138364FFF7EDFE060056F041012000FFF717FF6A
S11383746868401E000310F4E0412868401E0002AF
S113838410F470600143A868401E800110F0C0001E
S11383940143E868401E10F03F00014314F10C004F
S11383A4FFF7FDFEE868401E800910F00F0114F188
S11383B41800FFF7F4FE36F04006F00701D57608FE
S11383C4760031002000FFF7EAFE70BD38B50400E2
S11383D40D002000FFF78CFE002805D140F29251D5
S11383E4DFF86C0400F050FAEDB2002D05D0022D34
S11383F419D00CD3032D22D02DE0201DFFF79FFEAE
S113840405007FF01F01201DFFF7C9FE24E014F5C9
S11384148070FFF794FE050014F58270FFF78FFE59
S113842455EA004518E014F59070FFF788FE05003E
S113843414F59270FFF783FE55EA00450CE014F539
S1138444B070FFF77CFE050014F5B270FFF777FEF9
S113845455EA004500E00025280032BD2DE9FB4F14
S11384640400150000272000FFF742FE002805D170
S113847440F25F61DFF8D80300F006FA019821287E
S113848402D20198002805D14FF4CC61DFF8C0036F
S113849400F0FAF99DF80800002819D09DF80800A6
S11384A4012815D09DF80800022811D09DF8080071
S11384B403280DD09DF80800012809D09DF8080070
S11384C4042805D040F26661DFF8840300F0DCF987
S11384D414F12000FFF733FE0004F9D42868B0F542
S11384E4006F02D2287A400701D5012000E0002061
S11384F45FF0930B0021ADF8001000265FF0000A32
S11385045FF000085FF000099DF80810002906D008
S113851402291CD017D3042926D01AD32AE05AF4EA
S1138524807A4FF400560127297A09072BD5C0B263
S1138534002820D0D5F804806968090C5FEAC14991
S11385445FEAD9491FE05AF4807A0026ECE7002652
S1138554EAE74FF400564FF4805A4FF6FF7841F699
S1138564FF795BF0400BDFE74FF400564FF4905A69
S11385740127D9E783E05FF00008696889005FEAAE
S1138584C1495FEAD949297A11F02801282901D17E
S113859459F40049297A11F01801182901D159F420
S11385A48049297A11F0380F03D05AF4805A5BF0C9
S11385B4400B5BF0200BC0B200280DD0BDF80000C6
S11385C429680843ADF800002868000CC004C00CF6
S11385D4064356F4404606E028688000C004C00CF4
S11385E4064356F40046287B10F00F0050EA0A0AAA
S11385F4A868800501D45AF0800A287AC00701D5F6
S11386045AF4006A287A800701D55AF4806AFFB2C2
S1138614002F05D0EA6814F13C012869FFF7CCFD6A
S11386241FFA8BFB594614F12400FFF7B8FD1FFA17
S113863488F8414614F12800FFF7B1FD1FFA89F9BF
S1138644494614F12C00FFF7AAFDBDF8001014F1FB
S11386543000FFF7A4FDB6B2310014F13400FFF783
S11386649EFD1FFA8AFA514614F13800FFF797FD6C
S1138674019810F03F0114F12000FFF790FDBDE8CC
S1138684F78F2DE9F04704000D0016001F002000A9
S1138694FFF72EFD002804D140F2C1716C4800F0AC
S11386A4F3F8212D01D2002D04D140F2C27168489F
S11386B400F0EAF87321FFB2002F01D051F0080151
S11386C489B214F18400FFF76AFD15F03F0114F137
S11386D48000FFF764FD14F18000FFF730FD00040F
S11386E4F9D414F18800FFF72AFD070014F18C0073
S11386F4FFF725FD804614F19000FFF720FD814625
S113870414F19400FFF71BFD824614F19800FFF75F
S113871416FD0021B160C10502D45FEA8A4104D484
S1138724C10506D55FEA8A4103D4B16851F040011A
S1138734B1605FEA4A410ED51FFA8AFA464911EA42
S11387440A411FFA89F959EA01013160B16851F00B
S11387540401B16003E0CAF38A0189B231604104BF
S113876403D5B16851F48071B160C10435D55FEAB1
S11387744A4114D51FFA88F8374911EA0841BFB2AF
S11387843943716071687FF06042914202D1317A59
S1138794490614D4B16851F00801B1600FE0C8F37C
S11387A48A0189B27160716840F2FF72914202D108
S11387B4317A490603D4B16851F00801B1605FEA23
S11387C4084103D5B16851F02801B1605FEA48411A
S11387D403D5B16851F01801B160010503D5B1683E
S11387E451F00101B160410503D5B16851F00201B2
S11387F4B160010422D580B210F00F00F060307A29
S1138804400605D4F26814F19C013069FFF7E9FCD1
S1138814042114F18400FFF7C2FC15F03F0114F1A4
S11388248000FFF7BCFC14F18000FFF788FC00040F
S1138834F9D4B06850F08000B06001E00020F0602A
S1138844BDE8F08700000440001004400020044008
S1138854B899000004E100E00000FF1F80B500F0B7
S113886407F800F0A3F800F0C9F900F0A5F8FAE756
S113887480B5044800F0CAFA00F0B2F900F0F2FC42
S113888401BD00008003C001FEE7010010B504002F
S1138894472C04D34FF4D5713D48FFF7F5FF042C5E
S11388A406D13C48006850F480303A4908602DE011
S11388B4052C06D13748006850F400303549086067
S11388C424E0062C06D13348006850F48020314952
S11388D408601BE00F2C06D12F48006850F00200FA
S11388E42D49086012E0B4F11000202806D20120BA
S11388F4B4F1100188402949086007E0302C05D3FD
S11389040120B4F1300188402549086010BD10B538
S11389140400472C04D34FF4F7711D48FFF7B4FF48
S1138924042C06D11B48006830F4803019490860CF
S11389342DE0052C06D11748006830F400301549A1
S1138944086024E0062C06D11248006830F4802024
S1138954104908601BE00F2C06D10F48006830F062
S113896402000D49086012E0B4F11000202806D278
S11389740120B4F1100188400A49086007E0302C52
S113898405D30120B4F1300188400749086010BDC3
S11389949898000024ED00E010E000E000E100E01D
S11389A404E100E080E100E084E100E080B500F04F
S11389B40DF800F0B9F801BD80B500F01DF800F021
S11389C4D9F801BD80B500F016FA01BD80B5784828
S11389D400F0F1F9774800F0EEF903215FF040204C
S11389E400F0F5FD00F0C0FA60234FF46142010089
S11389F4714800F03CFE01BD80B570480078002841
S1138A0413D16F4800F03EF801283AD16C4800783D
S1138A14002836D000F03AFC6A490860012067490E
S1138A2408700020684908702BE065486649097895
S1138A340844401C00F026F8012818D16248007844
S1138A44401C61490870604800785D49097888428F
S1138A5417D100205949087059484078FF2810D18B
S1138A645748807800280CD1FFF7ACFF09E000F0E8
S1138A740DFC544909686431814202D200204F49F3
S1138A84087001BD10B504004B4800F0B7FE10F1A6
S1138A94010F02D02070012000E0002010BD00B5B9
S1138AA485B0042002901020009002E00098401E3B
S1138AB400900098002834D00820019002E0019826
S1138AC4401E019001980028F0D00098401C6421B5
S1138AD448430099019A5118491CB0FBF1F0C0B203
S1138AE441380B28EBD210200099019A5118491CE3
S1138AF4B0FBF1F201FB12000028E0D10198042834
S1138B0401D20198029010200099019A5118491C2D
S1138B14B0FBF1F0039069462C48FFF7DBFB01201E
S1138B2400E0002005B000BD00B585B0284800F081
S1138B3442F90321274800F013FD274800F03BF9CC
S1138B442248FFF762FBFFF7AAFF2048FFF7ACFBBC
S1138B5440F26760009040F2FF7001900820029098
S1138B640820039002236A4601211848FFF776FC83
S1138B7405B000BD00B587B002211448FFF726FCF8
S1138B8416490988084211D068460690012302AAAE
S1138B9401210E48FFF775FD9DF80000FF2805D15B
S1138BA49DF80100002801D1FFF70CFF07B000BDB8
S1138BB4010000100100002000C00040510000200A
S1138BC40000002044000020500000200000044065
S1138BD40800002000700040000110008E8800008E
S1138BE480B5174800F0E7F80121164800F0D4FCDA
S1138BF400220121134800F09EFC01BD10B500F0D1
S1138C0445FB040010480068201AB0F5FA7F16D317
S1138C140E480078002808D101200C49087001226C
S1138C240121084800F087FC07E000200749087088
S1138C3400220121034800F07EFC0348046010BDB7
S1138C442000002000500240480000205200002070
S1138C54DFF80C15884200F0A980DFF80815884273
S1138C6400F0A480DFF80015884200F09F80DFF84C
S1138C74FC14884200F09A80DFF8F414884200F06F
S1138C849580DFF8F014884200F09080DFF8E8144F
S1138C94884200F08B80DFF8E414884200F0868078
S1138CA4DFF8DC14884200F08180DFF8D8148842AD
S1138CB47CD0DFF8D414884278D0DFF8D01488420A
S1138CC474D0DFF8CC14884270D0DFF8C81488421A
S1138CD46CD0DFF8C414884268D0DFF8C01488422A
S1138CE464D0DFF8BC14884260D0DFF8B81488423A
S1138CF45CD0DFF8B414884258D0402856D0B0F180
S1138D04102F53D0DFF8A41488424FD0DFF8A014F6
S1138D1488424BD0DFF89C14884247D0DFF898147B
S1138D24884243D0DFF8941488423FD0B0F1101F36
S1138D343CD0DFF88C14884238D0DFF88814884299
S1138D4434D0DFF88414884230D0DFF880148842A9
S1138D542CD0DFF87C14884228D0DFF878148842B9
S1138D6424D0DFF87414884220D0DFF870148842C9
S1138D741CD0DFF86C14884218D0DFF868148842D9
S1138D8414D0DFF86414884210D0DFF860148842E9
S1138D940CD0B0F1202F09D0DFF85414884205D048
S1138DA4082803D0DFF85014884201D1012000E0E0
S1138DB40020C0B2704710B504002000FFF748FF3C
S1138DC4002805D14FF4FC71DFF82804FFF75CFD9B
S1138DD4DFF82804210F50F821000068A1B2220C06
S1138DE412F01F0291400843DFF81014220F51F8C7
S1138DF42210086010BDDFF81404DFF814140860AE
S1138E04FEE700000138FDD17047704770B50400D7
S1138E14DFF80004006810F0E04F08D0DFF8F40332
S1138E240068DFF8F4130840B0F1805F02D1002C2D
S1138E3400F19980DFF8C8030568DFF8E0030668E9
S1138E4455F4006535F4800556F40066DFF8B00384
S1138E540560DFF8C8030660A80701D5A00708D594
S1138E6415F0010014F0010191F00101C0B20842AF
S1138E741ED074F003000540DFF884030560002E5F
S1138E8407D516F07000302809D016F07000702849
S1138E9405D0002E08D415F03000302804D14FF446
S1138EA48050FFF7AFFF03E05FF40020FFF7AAFF51
S1138EB4DFF86C03054043F2F07020400543DFF80B
S1138EC464030640DFF8600320400643E00010F02A
S1138ED4400006434020DFF82C130860002E06D51A
S1138EE4DFF838030660DFF81803056005E0DFF8EF
S1138EF410030560DFF8240306601020FFF782FFE7
S1138F04DFF828030540DFF828032040054336F042
S1138F14FC5614F0FC500643600008D555F4800553
S1138F2436F48006DFF80C032040064301E036F0F3
S1138F34804620050ED44FF4004000E0401E002873
S1138F4404D0DFF8C41209684906F7D535F400657E
S1138F5436F40066DFF8A8020560DFF8C002066094
S1138F641020FFF74FFF70BD30B4DFF8940201689E
S1138F74DFF8A8020268002A02D512F0700001E0AA
S1138F8411F0300000280DD010283AD020286FD0DA
S1138F94302800F0A480602800F0A480702800F039
S1138FA4A480A5E0DFF89002C1F3841350F82300F1
S1138FB4DFF888321340B3F1004F05D0002A00F1E2
S1138FC4AA800B0500F1A780DFF874321B68DFF870
S1138FD44442246814F0E04F09D0DFF8384224688E
S1138FE4DFF834522C40B4F1805F40F08380C3F343
S1138FF44814A41C604313F01F04A41CB0FBF4F035
S113900481E0DFF81002006810F0E04F08D0DFF8C8
S113901404020068DFF800321840B0F1805F02D126
S1139024DFF8200223E0DFF8EC010068DFF8E83120
S11390341840DFF81432984205D1DFF8D8010068EB
S113904480B202280ED0DFF8CC010068DFF8C83102
S11390541840DFF8F831984207D1DFF8B801006806
S1139064000402D1DFF8E80101E0DFF8E8019FE73A
S1139074DFF8A001006810F0E04F08D0DFF8940195
S11390840068DFF894311840B0F1805F02D1DFF852
S1139094C80123E0DFF87C010068DFF87C31184064
S11390A4DFF8A431984205D1DFF86801006880B282
S11390B402280ED0DFF85C010068DFF85C31184048
S11390C4DFF88831984207D1DFF8480100680004CA
S11390D402D1DFF8880101E0DFF8840168E747F290
S11390E4305065E75FF4800062E74FF400405FE7C7
S11390F4002032E0C3F34814604313F01F04641CDB
S11391046400B0FBF4F05C0400D540081B0400D5F3
S1139114800851F480014B021FD5002A18D553004E
S113912410D5DFF818311340B3F1004F03D0002AEF
S113913408D4090506D44000C2F38651491CB0FB87
S1139144F1F00AE0C2F3C551491CB0FBF1F004E0AC
S1139154C1F3C351491CB0FBF1F030BC70470000AB
S113916401001000020010000001100000021000B1
S1139174000410000001101000021010000410106C
S113918400401010005010200100002002000020B4
S1139194040000200800002010000020200000200B
S11391A44000002080000020000100200040001046
S11391B40010101000011020800000301000003056
S11391C40001001000020010100000102000001024
S11391D420000030010010100200101004001010D0
S11391E40800101001000010020000100400001018
S11391F401001020F898000000101000F89B0000F3
S113920460E00F4058E00F4050E00F400400FA05BE
S11392140CED00E000E00F400000FF7070E00F4030
S11392240FC8FFFF8FDFFF7F30200080FCFF3FF873
S11392340300C00700004040709A0000000800804A
S113924464E00F40C0E1E4000000011000000310DA
S1139254001BB7000024F40070383900C0C62D0088
S113926400093D0080B5FFF77FFE4FF47A71B0FB2F
S1139274F1F000F0F9FA00F0E9FA00F0EEFA002057
S113928400F001F801BD064908607047044800680D
S1139294704703480068401C014908607047000097
S11392A44C000020B0F1402F43D0DFF8581388421B
S11392B43FD0DFF8541388423BD0DFF85013884280
S11392C437D0DFF84C13884233D0DFF84813884290
S11392D42FD0DFF8441388422BD0DFF840138842A0
S11392E427D0DFF83C13884223D0DFF838138842B0
S11392F41FD0DFF8341388421BD0DFF830138842C0
S113930417D0DFF82C13884213D0DFF828138842CF
S11393140FD0DFF8241388420BD0DFF820138842DF
S113932407D0DFF81C13884203D0DFF818138842EF
S113933401D1012000E00020C0B2704770B50400E0
S11393440D0016002000FFF7ADFF002804D1E4212E
S1139354DFF8F402FFF798FA002E08D0012E06D0A5
S1139364022E04D0E621DFF8E002FFF78DFAF007BD
S113937405D514F580600068EDB2284304E014F5C3
S113938480600068EDB2A84314F580610860B007FA
S113939405D514F584600068EDB2284304E014F59F
S11393A484600068EDB2A84314F58461086070BD5C
S11393B4F8B504000D0017001E002000FFF772FF2B
S11393C4002805D14FF4DD71DFF87C02FFF75CFA65
S11393D4012F0BD0022F09D0042F07D00C2F05D056
S11393E44FF4DF71DFF86002FFF74EFA082E11D054
S11393F40A2E0FD00C2E0DD0092E0BD00B2E09D013
S11394040D2E07D0002E05D040F2C511DFF8380226
S1139414FFF73AFAF80705D514F5A0600068EDB231
S1139424284304E014F5A0600068EDB2A84314F5E1
S1139434A0610860B80705D504F204500068EDB2D1
S1139444284304E004F204500068EDB2A84304F293
S113945404510860780705D514F5A1600068EDB2DD
S1139464284304E014F5A1600068EDB2A84314F5A0
S1139474A1610860380705D514F5A3600068EDB24E
S1139484284304E014F5A3600068EDB2A84314F57E
S1139494A3610860F00705D504F20C500068EDB22E
S11394A4284304E004F20C500068EDB2A84304F22B
S11394B40C510860B00705D514F5A2600068EDB23C
S11394C4284304E014F5A2600068EDB2A84314F53F
S11394D4A2610860700705D504F214500068EDB267
S11394E4284304E004F214500068EDB2A84304F2E3
S11394F414510860300705D504F21C500068EDB21D
S1139504284304E004F21C500068EDB2A84304F2BA
S11395141C510860002E05D114F5A5600068EDB255
S1139524284304E014F5A5600068EDB2A84314F5DB
S1139534A5610860F1BD70B504000D00160020009B
S1139544FFF7B0FE002805D14FF45171DFF8F8009D
S1139554FFF79AF9F6B2EDB214EB8500066070BD1C
S113956438B504000D002000FFF79CFE002805D147
S11395744FF46471DFF8D000FFF786F90222290062
S1139584C9B22000FFF7DAFE082304222900C9B275
S11395942000FFF70DFF31BD38B504000D00200095
S11395A4FFF780FE002804D140F204412648FFF767
S11395B46BF901222900C9B22000FFF7BFFE08237A
S11395C401222900C9B22000FFF7F2FE31BD38B5EB
S11395D404000D002000FFF765FE002804D140F2CA
S11395E41F511948FFF750F902222900C9B220007B
S11395F4FFF7A4FE082301222900C9B22000FFF7C3
S1139604D7FE31BD00800540005000400090054065
S11396140060004000A005400070004000B0054018
S11396240040024000C005400050024000D0054004
S11396340060024000E005400070024000F0054074
S113964400D0034000000640149A0000DFF8D8114B
S1139654884207D0DFF8D411884203D0DFF8D01150
S1139664884201D1012000E00020C0B27047F8B55F
S113967404000E0017001D002000FFF7E7FF002878
S113968405D140F20D11DFF8AC01FFF7FDF8002F0E
S113969405D14FF48771DFF89C01FFF7F5F8DFF883
S11396A49801006810F0E04F27D0DFF88C010068BF
S11396B4DFF888110840B0F1805F1ED0DFF878012C
S11396C40068DFF878110840DFF87411884205D186
S11396D4DFF86401006880B202280ED0DFF8580174
S11396E40068DFF858110840DFF85811884206D1A1
S11396F4DFF844010068000401D1102000E00820D0
S113970400FB07F0864205D240F20F11DFF8240172
S1139714FFF7BAF8200000F04DF8B6EB071F09D2A2
S113972414F13000006850F0200014F13001086096
S11397347F0807E014F13000006830F0200014F1D1
S113974430010860F000B0FBF7F0401C40088109C8
S113975414F12402116010F03F0014F12801086090
S113976414F12C000560002014F118010860200095
S113977400F001F8F1BD10B504002000FFF766FF06
S1139784002805D14FF4CF71DFF8A800FFF77CF867
S113979414F12C00006850F0100014F12C0108603E
S11397A414F13000006840F20131084314F130012F
S11397B4086010BD10B504002000FFF747FF00281F
S11397C405D14FF4DF71DFF86C00FFF75DF814F195
S11397D4180000680007FAD414F12C00006830F073
S11397E4100014F12C01086014F130000068DFF853
S11397F45810084014F13001086010BD10B504007D
S11398042000FFF723FF002804D140F2094109484E
S1139814FFF73AF814F118000068C00601D4206870
S113982401E05FF0FF3010BD00C0004000D00040F4
S113983400E00040CC9A000000E00F400000FF70FC
S11398440000011000000310FEFCFFFF0E48006836
S113985450F005000C49086070470B48006850F04C
S1139864020009490860704710B50400002C02D0B6
S1139874B4F1807F03D9D0210448FFF705F8601EB2
S11398840349086010BD000010E000E0589900008E
S113989414E000E0433A5C576F726B5C736F667458
S11398A4776172655C4F70656E424C545C546172AE
S11398B46765745C44656D6F5C41524D434D335F21
S11398C44C4D33535F454B5F4C4D3353383936322B
S11398D45F4941525C50726F675C6C69625C64728C
S11398E4697665726C69625C696E746572727570AE
S11398F4742E6300433A5C576F726B5C736F6674C7
S1139904776172655C4F70656E424C545C5461724D
S11399146765745C44656D6F5C41524D434D335FC0
S11399244C4D33535F454B5F4C4D335338393632CA
S11399345F4941525C50726F675C6C69625C64722B
S1139944697665726C69625C73797363746C2E6393
S113995400000000433A5C576F726B5C736F66746B
S1139964776172655C4F70656E424C545C546172ED
S11399746765745C44656D6F5C41524D434D335F60
S11399844C4D33535F454B5F4C4D3353383936326A
S11399945F4941525C50726F675C6C69625C6472CB
S11399A4697665726C69625C7379737469636B2E2E
S11399B463000000433A5C576F726B5C736F6674A8
S11399C4776172655C4F70656E424C545C5461728D
S11399D46765745C44656D6F5C41524D434D335F00
S11399E44C4D33535F454B5F4C4D3353383936320A
S11399F45F4941525C50726F675C6C69625C64726B
S1139A04697665726C69625C63616E2E6300000042
S1139A14433A5C576F726B5C736F667477617265FB
S1139A245C4F70656E424C545C5461726765745C3F
S1139A3444656D6F5C41524D434D335F4C4D33531C
S1139A445F454B5F4C4D3353383936325F4941528D
S1139A545C50726F675C6C69625C6472697665728F
S1139A646C69625C6770696F2E63000040420F008A
S1139A7400201C0080841E0000802500999E36006E
S1139A840040380000093D0000803E0000004B0007
S1139A94404B4C0000204E00808D5B0000C05D00F4
S1139AA40080700000127A0000007D008096980007
S1139AB4001BB7000080BB00C0E8CE00647ADA0063
S1139AC40024F4000000FA00433A5C576F726B5CA4
S1139AD4736F6674776172655C4F70656E424C5443
S1139AE45C5461726765745C44656D6F5C41524D8E
S1139AF4434D335F4C4D33535F454B5F4C4D3353B0
S1139B04383936325F4941525C50726F675C6C6914
S1139B14625C6472697665726C69625C75617274A4
S1139B242E63000019E050F8041BCB0744BFA9F1CD
S1139B3401035918121F0023042A41F8043BF9D2E3
S1139B445FEA827C0B4604D54FF0000CA1F800C0F8
S1139B549B1CD10744BF0021197050F8042B002A20
S1139B64E1D1704710B5074979441831064C7C4457
S1139B74163404E00A68081D114488470146A142CA
S1139B84F8D110BD080000001400000099FFFFFF85
S1139B9454000000000000200000000000F00BF856
S1139BA4002801D0FFF7DEFF0020AFF30080FEF7AA
S1139BB455FE00F002F80120704700F001B8FEE7FA
S1139BC40746384600F002F8FBE7000080B5AFF31F
S1139BD40080024A11001820ABBEFBE726000200F5
S1139BE4034B9D46AFF30080AFF30080FFF7D6FF2D
S1139BF45804002000E10F4004E10F4008E10F4045
S9039BE57C
